:020000000134C9
:2000340075817A758901D2AFD28C1206AD12001B80FB740A75F000C0E0C0F0740275F000E3
:20005400C0E0C0F01209C315811581158115815480C5F05400C5F045F07003020075020053
:2000740046740175F00022120046740A75F000C0E0C0F0740075F000C0E0C0F0740175F09C
:2000940000C0E0C0F01209EC7FFA122C11221200467BFF7CFF122D3845F070030200BB746E
:2000B400FF75F0FF020124740A75F000C0E0C0F0740075F000C0E0C0F0743875F000C0E095
:2000D400C0F01209EC7FFA122C11120046740A75F000C0E0C0F0740075F000C0E0C0F07465
:2000F4000C75F000C0E0C0F01209EC7FFA122C1112007B740075F000C0E0C0F0740075F0CD
:2001140000C0E0C0F012012515811581158115812212004678FB122C05E6122C379001E7E8
:20013400022C40740A75F000C0E0C0F0740075F000C0E0C0F078F5122C05E62480122C3732
:20015400C0E0C0F01209EC7FFA122C110201FB740A75F000C0E0C0F0740075F000C0E0C002
:20017400F078F5122C05E624C0122C37C0E0C0F01209EC7FFA122C110201FB740A75F0008C
:20019400C0E0C0F0740075F000C0E0C0F078F5122C05E62494122C37C0E0C0F01209EC7F39
:2001B400FA122C110201FB740A75F000C0E0C0F0740075F000C0E0C0F078F5122C05E624CE
:2001D400D4122C37C0E0C0F01209EC7FFA122C110201FBBB0103008F0102006301010037B8
:2001F4000100000000FB01220581740078FE122C05F678FE122C05E618181818860108860F
:200214000275F000122C2789828A83E493122C377B00122C2E122D4145F0700302028280E5
:200234000B78FE122C05E604F61480C6120046740A75F000C0E0C0F0740175F000C0E0C0E7
:20025400F078FA122C05E618181818860108860275F000122C2789828A83E493122C37C0FA
:20027400E0C0F01209EC7FFA122C1102023578FA122C05E60886F0158122120046740A75B6
:20029400F000C0E0C0F0740175F000C0E0C0F078F7122C05E6122C37C0E0C0F01209EC7FFD
:2002B400FA122C11227F08122C1178F3122C05E60886F07B007C00122D1845F070030202DD
:2002D400E8740075F00079F7122C0A122C27742DF70202F8740075F00079F7122C0A122CC9
:2002F40027742BF778F3122C05E60886F078FD122C05F608A6F078F3122C05E60886F07B42
:20031400007C00122D1845F0700302034678FD122C05E60886F0122D1178F3122C05F608EB
:20033400A6F018E60886F0122CFE18F608A6F0122D07740175F00079F7122C0A122C2778FA
:20035400F3122C05E60886F07BE87C03122C842430C5F03400C5F0F718E60886F07BE87C07
:2003740003122C7D78FD122C05F608A6F0740275F00079F7122C0A122C2778FD122C05E6C9
:200394000886F07B647C00122C842430C5F03400C5F0F778F3122C05E60886F07B647C0058
:2003B400122C7D78FD122C05F608A6F0740375F00079F7122C0A122C2778FD122C05E60883
:2003D40086F07B0A7C00122C842430C5F03400C5F0F7740475F00079F7122C0A122C277479
:2003F4002EF7740575F00079F7122C0A122C2778FD122C05E60886F07B0A7C00122C7D24CD
:2004140030C5F03400C5F0F7740075F00079F7122C0A122C27E7122C37C0E0C0F012028EBF
:2004340015811581740175F00079F7122C0A122C27E7122C37C0E0C0F012028E158115810B
:20045400740275F00079F7122C0A122C27E7122C37C0E0C0F012028E15811581740375F03A
:200474000079F7122C0A122C27E7122C37C0E0C0F012028E15811581740475F00079F71272
:200494002C0A122C27E7122C37C0E0C0F012028E15811581740575F00079F7122C0A122C5F
:2004B40027E7122C37C0E0C0F012028E158115817FF8022C207F08122C1178F3122C05E658
:2004D4000886F07B007C00122D1845F070030204F8740075F00079F7122C0A122C27742DFF
:2004F400F7020508740075F00079F7122C0A122C27742BF778F3122C05E60886F078FD12BD
:200514002C05F608A6F078F3122C05E60886F07B007C00122D1845F0700302055678FD1216
:200534002C05E60886F0122D1178F3122C05F608A6F018E60886F0122CFE18F608A6F0120A
:200554002D07740175F00079F7122C0A122C2778F3122C05E60886F07BE87C03122C842482
:2005740030C5F03400C5F0F718E60886F07BE87C03122C7D78FD122C05F608A6F074027552
:20059400F00079F7122C0A122C2778FD122C05E60886F07B647C00122C842430C5F03400C4
:2005B400C5F0F778F3122C05E60886F07B647C00122C7D78FD122C05F608A6F0740375F02B
:2005D4000079F7122C0A122C2778FD122C05E60886F07B0A7C00122C842430C5F03400C509
:2005F400F0F7740475F00079F7122C0A122C2778FD122C05E60886F07B0A7C00122C7D240A
:2006140030C5F03400C5F0F7740075F00079F7122C0A122C27E7122C37C0E0C0F012028EBD
:2006340015811581740175F00079F7122C0A122C27E7122C37C0E0C0F012028E1581158109
:20065400740275F00079F7122C0A122C27E7122C37C0E0C0F012028E15811581740375F038
:200674000079F7122C0A122C27E7122C37C0E0C0F012028E15811581740475F00079F71270
:200694002C0A122C27E7122C37C0E0C0F012028E158115817FF8022C20758E037481F5A8D4
:2006B400E5884401F5887400F53E7400F574740C75F000C0E0C0F0740075F000C0E0C0F015
:2006D400E53E122C37C0E0C0F01209EC7FFA122C11740075F000F53A85F03BF53885F039BC
:2006F4007400F56A7400F511747075F017F56485F065746475F000F55A85F05B796B7A004C
:20071400E98AF0C0E0C0F0746475F000C0E0C0F0122A0A1581158115811581121CF1121B9B
:20073400361200A2745675F031C0E0C0F01201FC15811581740075F000C0E0C0F0740175BD
:20075400F000C0E0C0F01201251581158115811581745F75F031C0E0C0F01201FC15811542
:200774008174F475F001C0E0C0F0122A3D1581158174BFF537E5114402F511121862748000
:2007940075F025C0E0C0F0122A5A1581158179A07A2DE98AF0C0E0C0F0122A7D1581158151
:2007B4001213821214751213E4121361121260120BB6121117120E7F120EF7120F3D121588
:2007D4004712178D121938121E08121BA2121E9F121EC8121FE11221BA122628120B8D12BC
:1B07F40017C612183012186212097F1211C312271B12278F121ADF0207B7229E
:07000300C0D0C0E002080FAD
:20080F00C0F0C083C082C000C001C002C003C004C005C006C007120843D007D006D005D0C9
:20082F0004D003D002D001D000D082D083D0F0D0E0D0D032740875F000C0E0C0F07402755C
:20084F00F000C0E0C0F01209C31581158115811581F54285F043740875F000C0E0C0F0747F
:20086F000175F000C0E0C0F01209C31581158115811581F54485F045E5448545F05410C57E
:20088F00F05400C5F0F53FE5448545F05420C5F05400C5F0F540E5448545F0540FC5F05483
:2008AF0000C5F0F54485F045E5448545F07B087C00122CDFF54485F045E5428543F0454427
:2008CF00C5F04545C5F0F54285F043E53F60030208F2E5428543F07BFF7CFF122C69F542F1
:2008EF0085F043E5407003020903740F75F027F54285F043E53E122C37C333C5F033C5F062
:20090F00794A7A00122C27E5428543F0F709A7F0E53E04F53E14E53E5403F53E740C75F0B0
:20092F0000C0E0C0F0740075F000C0E0C0F0E53E122C37C0E0C0F01209EC7FFA122C117404
:20094F000175F000C0E0C0F0122A3D15811581E53E122C377B00122C2E122D3845F070038F
:20096F0002097EE59054BFF590E5114480F51122E51675F0007B627C00122D3845F0700318
:20098F000209A779D17A30E98AF0C0E0C0F0122A7D158115811213822278FB122C05E6F5B0
:2009AF0013E513A2E09290A2E19291A2E29292A2E392932278F9122C05E6122C37C0E0C0F0
:2009CF00F01209A81581158178FB122C05E60886F0C0E0C0F0122AB9158115812278F712FB
:2009EF002C05E6122C37C0E0C0F01209A81581158178F9122C05E60886F0C0E0C0F008E6C7
:200A0F00122C37C0E0C0F0122ADA158115811581158122122AFA74D075F000C0E0C0F01231
:200A2F002B0F15811581740775F000C0E0C0F0122B0F15811581749075F000C0E0C0F012CE
:200A4F002B0F15811581122B0722122AFA74D075F000C0E0C0F0122B0F158115817400752B
:200A6F00F000C0E0C0F0122B0F15811581122B07122AFA74D175F000C0E0C0F0122B0F15DA
:200A8F008115817400F57A7400F515E51575F0007B067C00122D4B45F07003020AD28008DB
:200AAF00E51504F5151480E3E51579527A0075F000122C27C001C002122B39D007D000F609
:200ACF00020AAF7401F57AE51579527A0075F000122C27C001C002122B39D007D000F612B7
:200AEF002B0722122AFA74D075F000C0E0C0F0122B0F15811581740075F000C0E0C0F012B1
:200B0F002B0F15811581740075F000C0E0C0F0122B0F15811581743075F000C0E0C0F01254
:200B2F002B0F15811581741275F000C0E0C0F0122B0F15811581740375F000C0E0C0F0124F
:200B4F002B0F15811581742575F000C0E0C0F0122B0F15811581740775F000C0E0C0F01218
:200B6F002B0F15811581740075F000C0E0C0F0122B0F15811581122B0722120A5922E51667
:200B8F0075F0007B757C00122D3845F07003020BB579ED7A2FE98AF0C0E0C0F0122A7D1504
:200BAF0081158112138222E51675F0007B747C00122D3845F07003020C61746775F031C0BC
:200BCF00E0C0F0122A7D15811581120D18F50D743A75F000C0E0C0F0122A911581158112EA
:200BEF000D18F50C743A75F000C0E0C0F0122A9115811581120D18F50A122AFA74D075F04F
:200C0F0000C0E0C0F0122B0F15811581740075F000C0E0C0F0122B0F15811581E50A75F008
:200C2F0000C0E0C0F0122B0F15811581E50C75F000C0E0C0F0122B0F15811581E50D75F068
:200C4F0000C0E0C0F0122B0F15811581122B07121382227F09122C11740075F00078FD1279
:200C6F002C05F608A6F0122AA9C0E0C0F0122A911581158178FC122C05F67B0D7C00122D82
:200C8F004145F07003020CCA801678FD122C05E60886F0122CFE18F608A6F0122D0780C65E
:200CAF0078FD122C05E60886F079F6122C0A122C2778FC122C05E6F7020C9978FD122C05FA
:200CCF00E60886F079F6122C0A122C277400F778FD122C05E60886F07B007C00122D38454B
:200CEF00F07003020CFD74FF75F0FF020D1379F6122C0AE98AF0C0E0C0F0122B6D158115BF
:200D0F0081020D137FF7022C2005810581058105810581740075F00078FD122C05F608A68A
:200D2F00F078FD122C05E60886F07B027C00122D1845F07003020D8A801678FD122C05E6D3
:200D4F000886F0122CFE18F608A6F0122D0780D178FD122C05E60886F079FA122C0A122C72
:200D6F0027C001C002122AA9C0E0C0F0122A9115811581D007D000F6020D4978FD122C05DF
:200D8F00E60886F079FA122C0A122C277400F7740075F00079FA122C0A122C27E7C39430EE
:200DAF00122C377B04122C2E122CDFC0E0C0F0740175F00079F8122C0A122C27E7C39430F1
:200DCF00D004D0034BC5F04CC5F0122C377FFB022C2005810581058105810581740075F0A8
:200DEF000078FD122C05F608A6F078FD122C05E60886F07B027C00122D1845F07003020E74
:200E0F0053801678FD122C05E60886F0122CFE18F608A6F0122D0780D178FD122C05E60899
:200E2F0086F079FA122C0A122C27C001C002122AA9C0E0C0F0122A9115811581D007D000B5
:200E4F00F6020E1278FD122C05E60886F079FA122C0A122C277400F779FA122C0AE98AF0A6
:200E6F00C0E0C0F0122B6D158115817FFB022C20E51675F0007B697C00122D3845F0700396
:200E8F00020EF6748675F031C0E0C0F0122A7D15811581740075F000C0E0C0F01209A81577
:200EAF00811581740475F000C0E0C0F0120C627B647C00122C69C0E0C0F0122AE81581153E
:200ECF008115811581740475F000C0E0C0F0122AC815811581F56485F065E5648565F0F5AE
:200EEF006285F06312138222E51154087003020F3CE5628563F0122D07F56285F063122CFC
:200F0F00FEE5628563F07B007C00122D5245F07003020F3CE5648565F0F56285F063E511E0
:200F2F004404F5111225B8E51154DFF511220581E51714F51704E51775F0007B007C001204
:200F4F002D5245F070030211147464F517120A59740275F00079527A00122C27E775F0000A
:200F6F007B047C00122CED78FE122C05F6E675F0007B0A7C00122C69F6740275F0007952FE
:200F8F007A00122C27C001C002740275F00079527A00122C27E7540F78FC122C0526D0075D
:200FAF00D000F6740175F00079527A00122C27E775F0007B047C00122CED78FE122C05F6B7
:200FCF00E675F0007B0A7C00122C69F6740175F00079527A00122C27C001C002740175F038
:200FEF000079527A00122C27E7540F78FC122C0526D007D000F6740075F000C0E0C0F01239
:20100F0009A815811581740275F00079527A00122C27C001C002740075F000C0E0C0F012A1
:20102F002AB915811581D007D00086037C00122D3845F0602B740175F00079527A00122C52
:20104F0027C001C002740175F000C0E0C0F0122AB915811581D007D00086037C00122D3869
:20106F0045F070030210A3E5114408F511742C75F001F55A85F05B743D75F000C0E0C0F031
:20108F00E51175F000C0E0C0F0122ADA1581158115811581740275F00079527A00122C27A3
:2010AF00C001C002740275F000C0E0C0F0122AB915811581D007D00086037C00122D3845EA
:2010CF00F0602B740175F00079527A00122C27C001C002740375F000C0E0C0F0122AB91549
:2010EF00811581D007D00086037C00122D3845F07003021114E51154F7F511746475F00054
:20110F00F55A85F05B158122E51675F0007B647C00122D3845F070030211C2749E75F03192
:20112F00C0E0C0F0122A7D15811581120D18F50E742D75F000C0E0C0F0122A9115811581E2
:20114F00120D18F50F742D75F000C0E0C0F0122A9115811581120D18F510122AFA74D075CB
:20116F00F000C0E0C0F0122B0F15811581740475F000C0E0C0F0122B0F15811581E50E759B
:20118F00F000C0E0C0F0122B0F15811581E50F75F000C0E0C0F0122B0F15811581E51075FD
:2011AF00F000C0E0C0F0122B0F15811581122B0712138222E51675F0007B0D7C00122D3880
:2011CF0045F070030211EB79A07A2DE98AF0C0E0C0F0122A7D158115811213822278FB12B4
:2011EF002C05E6122C37C333C5F033C5F0794A7A00122C27E70987F07B0A7C00122C84F500
:20120F004885F04978FB122C05E6122C37C333C5F033C5F0794A7A00122C27E70987F07B91
:20122F000A7C00122C7DF54174BD75F031C0E0C0F0E5488549F0C0E0C0F0E541122C37C07B
:20124F00E0C0F0740375F0001227C67FFA122C1122E51675F0007B2F7C00122D3845F07088
:20126F0003021360120A5974C475F031C0E0C0F0740475F00079527A00122C27E775F00081
:20128F00C0E0C0F0740575F00079527A00122C27E775F000C0E0C0F0740675F00079527AA7
:2012AF0000122C27E775F000C0E0C0F0740475F0001227C67FF8122C1174D575F031C0E0FD
:2012CF00C0F0740275F00079527A00122C27E775F000C0E0C0F0740175F00079527A0012FD
:2012EF002C27E775F000C0E0C0F0740075F00079527A00122C27E775F000C0E0C0F0740459
:20130F0075F0001227C67FF8122C11121450740075F000C0E0C0F01211EC15811581740145
:20132F0075F000C0E0C0F01211EC15811581740275F000C0E0C0F01211EC158115817403D1
:20134F0075F000C0E0C0F01211EC1581158112138222E5985401700302137D122AA9C0E069
:20136F00C0F0122A9115811581F51602138174FFF5162279BB7A2DE98AF0C0E0C0F0122AAA
:20138F007D158115812205810581740075F00078FD122C05F608A6F078FD122C05E6088616
:2013AF00F078F9122C058603088604122D1845F070030213DF801678FD122C05E60886F0BA
:2013CF00122CFE18F608A6F0122D0780CB0213C615811581221213EB12142522E5608561B4
:2013EF00F0122CFEF56085F061122D07E5608561F0AB5AAC5B122D5B45F07003021424742A
:20140F000075F000F56085F061E5114440F511C2977405F51422E5115440700302144FE569
:20142F001414F51404E51475F0007B007C00122D3845F0700302144FD297E51154BFF51117
:20144F0022E5904440F590E511548075F0007B007C00122D3845F0700302146E021456E5C3
:20146F0011547FF51122308DFDC28D438CDC2205810581740175F000796B7A00122C27E7EB
:20148F0075F00078FD122C05F608A6F018E60886F07B087C00122CDF18F608A6F07400755F
:2014AF00F000796B7A00122C2778FD122C05E60886F04715811581227401256BF56BE4353B
:2014CF006CF56CE4356DF56D221214C7740275F000796B7A00122C27E775F000C0E0C0F0FF
:2014EF001209A81581158112147E221214C71214C7740275F000796B7A00122C27E775F064
:20150F0000C0E0C0F01209A81581158112147E2278FB122C05E675F0007B047C00122CED90
:20152F00F62430C5F03400C5F02278FB122C05E6540F2430122C3722E511540470030217CE
:20154F0030121450120A591214FAC0E0C0F0E55E855FF0C0E0C0F0122AE8158115811581A4
:20156F0015811214D8C0E0C0F0740475F00079527A00122C27E775F000C0E0C0F0122ADA3F
:20158F0015811581158115811214D8C0E0C0F0740575F00079527A00122C27E775F000C002
:2015AF00E0C0F0122ADA15811581158115811214D8C0E0C0F0740675F00079527A00122C6E
:2015CF0027E775F000C0E0C0F0122ADA15811581158115811214D8C0E0C0F0740275F000A2
:2015EF0079527A00122C27E775F000C0E0C0F0122ADA15811581158115811214D8C0E0C0CA
:20160F00F0740175F00079527A00122C27E775F000C0E0C0F0122ADA15811581158115813D
:20162F001214D8C0E0C0F0740075F00079527A00122C27E775F000C0E0C0F0122ADA158182
:20164F001581158115811214FAC0E0C0F0740075F000794A7A00122C27E70987F0C0E0C007
:20166F00F0122AE815811581158115811214FAC0E0C0F0740275F000794A7A00122C27E71B
:20168F000987F0C0E0C0F0122AE815811581158115811214FAC0E0C0F0740475F000794ADF
:2016AF007A00122C27E70987F0C0E0C0F0122AE815811581158115811214FAC0E0C0F07425
:2016CF000675F000794A7A00122C27E70987F0C0E0C0F0122AE81581158115811581E511C5
:2016EF0054FBF511E55E855FF0122CFEF55E85F05F121731740075F000C0E0C0F01209A8C6
:20170F0015811581740675F000C0E0C0F0E55E855FF0C0E0C0F0122AE815811581158115FD
:20172F008122740075F000C0E0C0F01209A815811581743E75F000C0E0C0F0122AC81581DE
:20174F001581AB5EAC5F122D4B45F0700302178CE51154F7F511746475F000F55A85F05B56
:20176F00743C75F000C0E0C0F074FF75F0FFC0E0C0F0122ADA158115811581158122E51643
:20178F0075F0007B727C00122D3845F070030217C574E575F031C0E0C0F0E55E855FF0C059
:2017AF00E0C0F0740275F0001227C6158115811581158112138222740E75F000C0E0C0F058
:2017CF00740075F000C0E0C0F01209C315811581158115817BFF7C00122D4145F0600EE59D
:2017EF0011540175F0007B007C00122D3845F0700302182BE5114401F511740E75F000C0CC
:20180F00E0C0F0740075F000C0E0C0F01209C31581158115811581F53702182F74FFF537B6
:20182F0022740E75F000C0E0C0F0740075F000C0E0C0F01209C315811581158115817BFF67
:20184F007C00122D3845F07003021861E51154FEF51122E53775F0007BFF7C00122D4145B7
:20186F00F07003021937E53775F000901923022C40E57404F57414021937E5116402F5115B
:20188F00E51154EFF51112007B740075F000C0E0C0F0740175F000C0E0C0F012012515814C
:2018AF0015811581158174FB75F031C0E0C0F01201FC15811581E511540270030218E17499
:2018CF002075F000C0E0C0F012028E1581158102191A12007B12268F740075F000C0E0C094
:2018EF00F0740075F000C0E0C0F01201251581158115811581740075F032C0E0C0F01201C2
:20190F00FC15811581E5114410F5110219370219370219372019EF001D19DF008918BF00AD
:20192F0080187F000000371922E51675F0007B737C00122D3845F07003021ADE740075F053
:20194F0000C0E0C0F01209A815811581740975F032C0E0C0F0740075F000C0E0C0F0122A70
:20196F00B915811581C0E0C0F0740175F000C0E0C0F0122AB915811581C0E0C0F07403759C
:20198F00F0001227C67FFA122C11740075F000C0E0C0F0120DE1122C37C0E0C0F0122ADA7D
:2019AF001581158115811581743A75F000C0E0C0F0122A9115811581740175F000C0E0C02A
:2019CF00F0120DE1122C37C0E0C0F0122ADA1581158115811581741C75F032C0E0C0F074EA
:2019EF000275F000C0E0C0F0122AB915811581C0E0C0F0740375F000C0E0C0F0122AB9157A
:201A0F00811581C0E0C0F0740375F0001227C67FFA122C11740275F000C0E0C0F0120DE182
:201A2F00122C37C0E0C0F0122ADA1581158115811581743A75F000C0E0C0F0122A9115819E
:201A4F001581740375F000C0E0C0F0120DE1122C37C0E0C0F0122ADA158115811581158182
:201A6F00742F75F032C0E0C0F0740075F000C0E0C0F0122AB915811581C0E0C0F074017549
:201A8F00F000C0E0C0F0122AB915811581C0E0C0F0740275F000C0E0C0F0122AB9158115BB
:201AAF0081C0E0C0F0740375F000C0E0C0F0122AB915811581C0E0C0F0740575F000122792
:201ACF00C67FF6122C11121B3612268F12138222E51675F0007B6D7C00122D3845F0700397
:201AEF00021B35740075F000C0E0C0F01209A815811581744575F032C0E0C0F0740175F0F3
:201B0F00001227C615811581743E75F000C0E0C0F0120C62C0E0C0F0122AE81581158115EF
:201B2F0081158112138222740075F000C0E0C0F01209A815811581740075F000C0E0C0F075
:201B4F00122AB9158115817B637C00122D3845F07003021B84743C75F000C0E0C0F0740161
:201B6F0075F000C0E0C0F0122ADA1581158115811581021BA1743C75F000C0E0C0F074FF9D
:201B8F0075F0FFC0E0C0F0122ADA158115811581158122E51675F0007B3D7C00122D3845A2
:201BAF00F07003021CF0740075F000C0E0C0F01209A815811581746775F032C0E0C0F07457
:201BCF000075F000C0E0C0F0122AB915811581C0E0C0F0740175F000C0E0C0F0122AB9159C
:201BEF00811581C0E0C0F0740375F0001227C67FFA122C11747975F032C0E0C0F07402750D
:201C0F00F000C0E0C0F0122AB915811581C0E0C0F0740375F000C0E0C0F0122AB915811538
:201C2F0081C0E0C0F0740375F0001227C67FFA122C11748B75F032C0E0C0F0740475F0005E
:201C4F00C0E0C0F0122AC8158115817B647C00122C84C0E0C0F0740275F0001227C6158118
:201C6F0015811581158174A975F032C0E0C0F0743E75F000C0E0C0F0122AC815811581C038
:201C8F00E0C0F0740275F0001227C61581158115811581743C75F000C0E0C0F0122AB91504
:201CAF008115817B017C00122D3845F07003021CD874C075F032C0E0C0F0740175F00012EA
:201CCF0027C615811581021CED74C975F032C0E0C0F0740175F0001227C615811581121383
:201CEF008222740075F000C0E0C0F01209A815811581743D75F000C0E0C0F0122AB9158128
:201D0F001581F511740475F000C0E0C0F0122AC815811581F56485F065E5648565F0F5620E
:201D2F0085F063740675F000C0E0C0F0122AC815811581F55E85F05F79717A00E98AF0C0AF
:201D4F00E0C0F0742E75F000C0E0C0F0122A0A1581158115811581796E7A00E98AF0C0E08B
:201D6F00C0F0E55E855FF0C0E0C0F0122A0A1581158115811581796E7A00E98AF0C0E0C07B
:201D8F00F079717A00E98AF0C0E0C0F012295C1581158115811581796E7A00E98AF0C0E0DA
:201DAF00C0F0746475F000C0E0C0F0122A0A158115811581158179767A00E98AF0C0E0C00D
:201DCF00F0796E7A00E98AF0C0E0C0F012291B1581158115811581796B7A00E98AF0C0E0E1
:201DEF00C0F079767A00E98AF0C0E0C0F01229CD158115811581158122E51675F0007B6E3D
:201E0F007C00122D3845F07003021E9E74D075F032C0E0C0F0122A7D15811581122AA97BEA
:201E2F00797C00122D3845F07003021E9BE51154F7F511740075F000F55E85F05F74007594
:201E4F00F000C0E0C0F01209A815811581740675F000C0E0C0F0740075F000C0E0C0F012DA
:201E6F002AE81581158115811581796B7A00E98AF0C0E0C0F0746475F000C0E0C0F0122A0F
:201E8F000A158115811581158112244E12138222E51675F0007B3F7C00122D3845F07003CF
:201EAF00021EC779BF7A2DE98AF0C0E0C0F0122A7D1581158112138222E51675F0007B63AE
:201ECF007C00122D3845F07003021F85120A5974E375F032C0E0C0F0740475F00079527ADD
:201EEF0000122C27E775F000C0E0C0F0740575F00079527A00122C27E775F000C0E0C0F0AE
:201F0F00740675F00079527A00122C27E775F000C0E0C0F0740475F0001227C67FF8122CFC
:201F2F001174F475F032C0E0C0F0740275F00079527A00122C27E775F000C0E0C0F074019C
:201F4F0075F00079527A00122C27E775F000C0E0C0F0740075F00079527A00122C27E775E8
:201F6F00F000C0E0C0F0740475F0001227C67FF8122C11121382221214FAC0E0C0F0122AFB
:201F8F00C815811581F54885F049E5488549F07B0A7C00122C7DF541E5488549F07B0A7C7A
:201FAF0000122C84F54885F049740475F033C0E0C0F0E5488549F0C0E0C0F0E541122C371F
:201FCF00C0E0C0F0740375F0001227C67FFA122C1122E51675F0007B617C00122D3845F079
:201FEF0070030221B97400F575122522796E7A00E98AF0C0E0C0F0740175F000C0E0C0F00E
:20200F00122A0A1581158115811581796B7A00E98AF0C0E0C0F0796E7A00E98AF0C0E0C0DE
:20202F00F012292E1581158115811581796E7A00E98AF0C0E0C0F0796B7A00E98AF0C0E06B
:20204F00C0F01229CD1581158115811581796B7A00E98AF0C0E0C0F0746475F000C0E0C0B3
:20206F00F0122A0A1581158115811581740075F000F56885F069E5688569F0AB5EAC5F125E
:20208F002D4B45F0600CE57575F0007B007C00122D3845F070030221B68012E5688569F0AD
:2020AF00122CFEF56885F069122D0780C9740D75F000C0E0C0F012243C15811581740A7544
:2020CF00F000C0E0C0F012243C158115811214FAC0E0C0F0122AC815811581740B75F0335C
:2020EF00C0E0C0F0E5688569F0C0E0C0F0740275F0001227C61581158115811581740F75DC
:20210F00F033C0E0C0F01214D8C0E0C0F0122AB915811581C0E0C0F01214D8C0E0C0F0121E
:20212F002AB915811581C0E0C0F01214D8C0E0C0F0122AB915811581C0E0C0F0740475F095
:20214F00001227C67FF8122C11741F75F033C0E0C0F01214D8C0E0C0F0122AB915811581C1
:20216F00C0E0C0F01214D8C0E0C0F0122AB915811581C0E0C0F01214D8C0E0C0F0122AB9FE
:20218F0015811581C0E0C0F0740475F0001227C67FF8122C11121F86121F86121F86121FBC
:2021AF00861223DB0220AA12138222E51675F0007B787C00122D3845F070030223DA1225C1
:2021CF0022796E7A00E98AF0C0E0C0F0740175F000C0E0C0F0122A0A1581158115811581F2
:2021EF00796B7A00E98AF0C0E0C0F0796E7A00E98AF0C0E0C0F012292E158115811581156B
:20220F0081796E7A00E98AF0C0E0C0F0796B7A00E98AF0C0E0C0F01229CD1581158115813F
:20222F001581796B7A00E98AF0C0E0C0F0746475F000C0E0C0F0122A0A158115811581153E
:20224F0081740075F000F56885F069E5688569F0AB5EAC5F122D4B45F070030223D78012DB
:20226F00E5688569F0122CFEF56885F069122D0780D9740D75F000C0E0C0F012243C1581D0
:20228F001581740A75F000C0E0C0F012243C158115811214FAC0E0C0F0122AC81581158128
:2022AF00742F75F033C0E0C0F0E5688569F0C0E0C0F0740275F0001227C61581158115816D
:2022CF0015811214D8C0E0C0F0122AB9158115811214D8C0E0C0F0122AB915811581121455
:2022EF00D8C0E0C0F0122AB9158115811214D8C0E0C0F0122AB9158115811214D8C0E0C0B9
:20230F00F0122AB9158115811214D8C0E0C0F0122AB915811581743375F033C0E0C0F0128D
:20232F0014FAC0E0C0F0122AC815811581C0E0C0F0740275F0001227C615811581158115FF
:20234F0081743775F033C0E0C0F01214FAC0E0C0F0122AC815811581C0E0C0F0740275F08F
:20236F00001227C61581158115811581743B75F033C0E0C0F01214FAC0E0C0F0122AC815D7
:20238F00811581C0E0C0F0740275F0001227C61581158115811581743F75F033C0E0C0F0FA
:2023AF001214FAC0E0C0F0122AC815811581C0E0C0F0740275F0001227C615811581158182
:2023CF0015811223DB02226F121382220581122BB178FE122C05F6E6122C377B1B122C2E6C
:2023EF00122D3845F070030223FD7401F57578FE122C05E6122C377B13122C2E122D3845E4
:20240F00F0700302243978FE122C05E6122C377B11122C2E122D4145F07003022439122B1B
:20242F00B178FE122C05F602241515812278FB122C05E6F5133099FDC299E513F599227459
:20244F004375F033C0E0C0F0122A7D1581158179187A00E98AF0C0E0C0F0741E75F000C0E8
:20246F00E0C0F0122BC31581158115811581740075F000C0E0C0F01209A8158115817400D9
:20248F0075F000F56885F069E5688569F079187A00122C27E775F0007B007C00122D4145EA
:2024AF00F070030224FC8012E5688569F0122CFEF56885F069122D0780CEE5688569F02471
:2024CF0008C5F03400C5F0C0E0C0F0E5688569F079187A00122C27E775F000C0E0C0F012AE
:2024EF002ADA15811581158115810224B7E5688569F02408C5F03400C5F0C0E0C0F07400DB
:20250F0075F000C0E0C0F0122ADA1581158115811581220581740D75F000C0E0C0F0122475
:20252F003C15811581740A75F000C0E0C0F012243C15811581740075F000C0E0C0F012090F
:20254F00A815811581740075F000F56885F069E5688569F02408C5F03400C5F0C0E0C0F03F
:20256F00122AB91581158178FE122C05F67B007C00122D4145F070030225B58012E568851D
:20258F0069F0122CFEF56885F069122D0780C078FE122C05E6122C37C0E0C0F0122A911590
:2025AF0081158102258C158122E51154F7F511746475F000F55A85F05B22E56A04F56A1201
:2025CF002C377B32122C2E122D2845F0700302261F7400F56AE53A853BF0F53885F039E5B8
:2025EF00B054087003022604740175F000F53A85F03B02260E740075F000F53A85F03BE595
:20260F003A853BF0C39538C5F09539C5F0022627740075F00002262722740075F000C0E0E7
:20262F00C0F01209A815811581743C75F000C0E0C0F0122AB9158115817B017C00122D38F7
:20264F0045F0700302268EE5B0540875F0007B007C00122D3845F0700302267EE5114408B9
:20266F00F511742C75F001F55A85F05B02268EE51154F7F511746475F000F55A85F05B22A5
:20268F00740075F000C0E0C0F01209A815811581743C75F000C0E0C0F0122AB9158115818D
:2026AF007B017C00122D3845F070030226ED740775F000C0E0C0F0740175F000C0E0C0F085
:2026CF001201251581158115811581744D75F000C0E0C0F012028E1581158102271A740759
:2026EF0075F000C0E0C0F0740175F000C0E0C0F01201251581158115811581744175F00042
:20270F00C0E0C0F012028E1581158122E5115402700302278E121450740075F000C0E0C045
:20272F00F0740075F000C0E0C0F01201251581158115811581E5745403F574E574243175A5
:20274F00F000C0E0C0F012028E15811581743D75F000C0E0C0F012028E15811581E574755A
:20276F00F000C333C5F033C5F0794A7A00122C27E70987F0C0E0C0F01202B9158115812253
:20278F00E511541070030227C5740075F000C0E0C0F0740175F000C0E0C0F012012515814E
:2027AF00158115811581E55E855FF0C0E0C0F01204C9158115812223F42581F88682088669
:2027CF008308E4FEFF93700122B42555A3E493B42D06430780A3E493B4300343074024D0E0
:2027EF00B40A00500CCE75F00AA42EFEA3E49380EDE493B46413E60886F030F7084307207D
:20280F00122D0EA6F018F68003B4750543070A801CB478054307108014B46F0B43070880F8
:20282F000C122A97A3809BB462624307027A00C004C005C006C007AB0753031F7C00E60807
:20284F0086F0122CACA6F018F6EDD007D006D005D0042430B43A0040022407C0E00AE6459E
:20286F00F070CCA902EF30E506742D122A970A1228FCD0E0122A97D9F90808EF30E7A5EABA
:20288F00C39E50A07420122A970A80F3B4630BAA011228FCE6122A9780DFB4732BC082C085
:2028AF008386820886837A00E4936004A30A80F886831886821228FCE493A36005122A9742
:2028CF0080F6D083D08280B1B4691986017A00E76004090A80F91228FC8601E7609B122AB4
:2028EF00970980F7F97A011228FCE980A8EE601B8FF020F716C002EAC39E500D742030F6BE
:20290F00027430122A970A80EED00222122A277A04C3E637F60809DAF9E4F5F092E02212B9
:20292F002A277A04C3E697F60809DAF980EB122A1FC37A04E633F608DAFA80DD122A1F7A7B
:20294F0004C82AC8C318E613F6DAFA80CC122A27AB00A8817F04122C1108AC001229D012E6
:20296F002A33A80312294E50077876A90412291EA8031229DC600CA804122940A804122930
:20298F00DC70DFA80379761229D07FFC022C20122A27AB00AC01122A337D21C3A80312291E
:2029AF0041DD02803378761229417876A9041229EB20E7E77876A904122931D380DE122AA8
:2029CF00277A04E7F60908DAFA22122A1F7A0475F000E6700308DAFA22122A277A04E82AD7
:2029EF00F8E92AF9181987F0E6B5F006DAF6E4F5F02274FF40F904F5F00422E58124FBF997
:202A0F008700122A3587000909E7F60809E7F622E58124FBF8860022E58124FBF8860118E8
:202A2F001886002278767A04760008DAFB2278FB122C058603088604BB0004BC00012279FE
:202A4F00E5A3D9FD1BBBFFF01C80F478FB122C058603088604748075F070122CAC122D0EE3
:202A6F00758921F58DF58B7588597598522278FB122C058682088683E493602D122A97A306
:202A8F0080F678FB122C05E63099FDC299F599B40A17740D80F2E430980C3098FDC298E5E2
:202AAF0099B40D02740A75F0002278FB122C058682088683E075F0002278FB122C058682B2
:202ACF00088683E0F5F0A3E0C5F02278F9122C05868208868308E6F02278F9122C0586822E
:202AEF0008868308E608F0A3E6F022D295122B5FC295122B65C29422C295122B5FD2952245
:202B0F0078FB122C05E67F0830E704D2958002C295122B5F23C294DFEFD295122B5F30957D
:202B2F0000122B65C294122B65227F087400D295122B5FA29533C294DFF6C0E0D295E57AD1
:202B4F00B40002C295122B5FC294D0E075F00022D2943094FD22000022000000002278FB30
:202B6F00122C058601E4FBFCFFE709B42D030FE709C39430B40A005012FA740A75F0001239
:202B8F002C692AFBE5F03400FC80E4EB8CF0DF03022D0E2278FB122C05E63099FDC299F5A9
:202BAF00992274FFF5F030980A3098FDC298E59975F0002278FB122C05860418188601E422
:202BCF00FD122AA9B408028003B47F16ED60F21D7408122A977420122A977408122A971900
:202BEF0080DF122A97F724F36006090DEDB504D1E4F7F5F0ED22C82581C822C92581C97ABA
:202C0F000022D083D082CF2581F581CFC082C08322CF2581F581CF2229F9E5F03AFA227CD8
:202C2F0000CB30E7011CCB2275F00030E70215F022FDE493A3FEE493A3FF4E7009E493FE8A
:202C4F00740193FF800BE493A3B5050BE493B5F0068F838E82E473A380D8FEEBA4FD8EF056
:202C6F00ECA4FCEB8EF0A4C5F02C2DC5F022122CAC8EF0ED22C0F0C0E0E5F06C5480FF8C60
:202C8F00F030F707EB122D0EACF0FBD0E0D0F030F703122D0EBF8005122CAC8062C002C0BF
:202CAF0001AAF0F97E007D007F11C3E933F9EA33FADF08F5F0E9D001D00222ED33FDEE333F
:202CCF00FEC3ED9BF5F0EE9C40E0ADF0FED380DBBB000122C333C5F033C5F0DBF722BB0024
:202CEF000122C3C5F013C5F013DBF722122CFE04700205F022122D0714B4FF0215F022124A
:202D0F002D07F4C5F0F4C5F022122D6B4029801E122D6B40227017801E122D6B4010701799
:202D2F00800C122D6B50108005122D7F6009E4F5F022122D7F60F7E4F5F00422122D7F4055
:202D4F00F680EB122D7F40EF70E480EB122D7F40DD70E480D9122D7F50DD80D2C39BC5F07F
:202D6F009C20E70720D207C345F02220D2F9D322C5F0C39C7003E5F09B22FBE493CB22FC33
:202D8F00E493FB740193CC22FAE493F9740193CA220A0A4D696E694C4F4747455220563354
:202DAF002E3320283F2068656C7029000A3E3E000A0A48454C50204D454E55202020202072
:202DCF0020202020202020202020200A2F207072696E7420616E616C6F6720726561646947
:202DEF006E67202020202020202020202020202020200A742054494D452073657420202056
:202E0F00202020202020202020202020200A642044415445207365742020202020202020EB
:202E2F0020202020202020200A6320436C6F636B20646973706C61792020202020202020F4
:202E4F0020202020202020200A73207365742053544152542F53544F50207265636F7264B8
:202E6F00696E672074696D65202020202020202020202020202020200A692073616D706C86
:202E8F00696E6720496E74657276616C202020202020202020202020202020200A3D2064B5
:202EAF006973706C61792073657474696E6720706172616D6574657273202020202020201F
:202ECF002020202020202020200A72206E756D626572206F66207265636F7264202020208A
:202EEF002020202020202020202020200A6D20736574206D6178696D756D207265636F7207
:202F0F0064202020202020202020202020202020200A62207465726D696E616C20636F6EF6
:202F2F006E656374696F6E202020202020202020202020202020200A6E204E6577207265D9
:202F4F00636F7264202020202020202020202020202020200A6120414C4C20726561643A60
:202F6F002070726573732045534320746F2073746F70202020202020202020202020202051
:202F8F0020200A78205265616420416C6C3A2073616D706C6520616E642064617461202062
:202FAF0020202020202020202020202020200A752041626F7574204D696E694C4F4747458D
:202FCF00522056332E31202020202020202020202020202020200A3F2068656C70000A4D1F
:202FEF00696E694C4F474745522077617320646573696E6765642062792057696368697471
:20300F00205349524943484F5445203238204A756E65203230303320202020202020202096
:20302F0020202020202020200A4170706C696564205068797369637320446570742E204B6F
:20304F004D49544C20202020202020202020202020202020200A6669726D7761726520750F
:20306F007064617465643A20323220417072696C20323030352020202020202020202020B2
:20308F002020202020200A55524C3A207777772E6B6D69746C2E61632E74682F7E6B737758
:2030AF00696368697420656D61696C3A206B73776963686974406B6D69746C2E61632E7413
:2030CF0068000A20312020202032202020203320202020342020202035202020203620205A
:2030EF00202037202020203820202020392020203130202031312020313220202020202013
:20310F0020202020202020202020202020200A494E312B20494E312D20494E322B20494E03
:20312F00322D20494E332B20494E332D20494E342B20494E342D202D3556202B35562020D9
:20314F00305620202B56004D696E694C4F47470045522056332E33000A656E746572206317
:20316F00757272656E742074696D652048483A4D4D3A5353203E000A20696E7465727661EC
:20318F006C20312D36303020736563203E20000A656E7465722063757272656E7420646197
:2031AF0074652044442D4D4D2D5952203E002025642E2564000A253032782D253032782DC0
:2031CF00253032782000253032783A253032783A2530327820000A2575207265636F7264ED
:2031EF007320617661696C61626C6500206D5620005265636F72643D20000A535441525435
:20320F0020253032643A25303264203E000A53544F502020253032643A25303264203E0013
:20322F000A20253032643A2530326420253032643A25303264000A456E746572206D6178A7
:20324F00696D756D207265636F7264732028312D3530303029203E000A205374617274204B
:20326F00253032643A25303264000A2053746F702020253032643A25303264000A20536131
:20328F006D706C696E6720496E74657276616C2873656329203D202575000A204D617869D7
:2032AF006D756D205265636F726473203D202575000A204D414E55414C000A204155544F5C
:2032CF00000A204E6577207265636F72643F28592F4E29000A253032782D253032782D25FF
:2032EF003032782000253032783A253032783A2530327820002025642E256400202564002B
:20330F0020253032782D253032782D253032780020253032783A253032783A253032780096
:20332F0020256400202564002025640020256400202564000A3C2D2D20456E7465722064EF
:20334F0065736372697074696F6E207465787420286D6178203330206368617261637465CD
:08336F007273292D2D3E0A00A6
:00000001FF
